:100000000C942A001895000018950000189500001F
:10001000189500001895000018950000189500002C
:10002000189500001895000018950000189500001C
:10003000189500001895000018950000189500000C
:1000400018950000189500001895000018950000FC
:10005000189500008FE58DBFC0E4E0E44E2E88E0E7
:100060008EBFD8E0F8E05F2EEEEFF7E0A0E6B0E05C
:1000700088278D933197E9F766248CEF84BB0E9423
:100080004E158E9A8D9A8C9A8F9AA09AA198A298C2
:100090008B98899A80E08ABBAEE2B1E0EEE0F7E3AC
:1000A0000E943B16A99AAA9A959894989698979A1E
:1000B000A89A8FEF809362000EE813EE28E33EE0EB
:1000C000ADE6B0E00D931D932D933C9301EC16E14A
:1000D0002CE631E0A1E7B0E00D931D932D933C9306
:1000E0000DEA18E624E230E0A5E7B0E00D931D9399
:1000F0002D933C9301E114EA23E030E0A9E7B0E05E
:100100000D931D932D933C9305E31DE520E030E016
:10011000ADE7B0E00D931D932D933C93EEECF4E22C
:100120008E2E9F2E81E080930C0100910C010133F3
:1001300018F011F00C94B600E82DF92DACE0B1E008
:10014000AD90BB24A5EEB1E0AA0CBB1CAA0CBB1C55
:10015000AA0DBB1D0E944A188E2E9F2EACE0B1E066
:100160008C918F5F8C9311F00C94950081E08093BB
:10017000D8010091D8010A3018F011F00C94CA008F
:100180000E947F0BA8EDB1E08C918F5F8C9311F0F2
:100190000C94B9005A924A9284E690E0A42DB52DB1
:1001A0008D939C9382E00E948A135A924A9281E036
:1001B000A42DB52D8C9381E00E948A130E942312F6
:1001C000249683E00E9486130E9420095A924A9244
:1001D00084E690E0A42DB52D8D939C9382E00E943F
:1001E0008A135A924A9281E0A42DB52D8C9381E016
:1001F0000E948A130E942312249683E00E94861391
:100200008FEF8BBB8AEF90E00E94441481E08093D3
:10021000D4010091D401033718F011F00C9422019D
:1002200088E0A4EDB1E0AD90BB24ACE5B1E0AA0D4F
:10023000BB1D8C93A4EDB1E08C918F5F8C9311F07A
:100240000C94090104E71EE020E030E0A1E8B0E0F2
:100250000D931D932D933C9384E08093AF00809188
:10026000D7018F7D8093D701ECEEF5E2AFEAB0E0E5
:100270008C919927A5E8B0E00E94541883E0809300
:10028000AE00E2E9F5E2AEEAB0E08C919927A9E888
:10029000B0E00E945418EAEBF5E283E00E945B189C
:1002A000A9EAB0E00E943B160E9416060E94BF0613
:1002B000A5E8B0E00D911D912D913C9142E050E0F8
:1002C00060E070E00E94E713ADE9B0E04D935D930C
:1002D0006D937D93A1E8B0E00D911D912D913C911E
:1002E000ADE9B0E04D915D916D917C910E94FC185B
:1002F000ADE8B0E00D931D932D933D93E2EDF6E351
:100300000E942018E5E8F0E00E94BA160E94DE166E
:100310000E942F17FF27EDE0A5E9B0E00E947519B4
:100320000027A7EDB1E08C9185FB0EF401E040E0E1
:10033000041711F00C94AA01ADE8B0E00D911D91E5
:100340002D913C91A1EBB0E00D931D932D933C9327
:100350000C94B601A1E8B0E00D911D912D913C9156
:10036000A1EBB0E00D931D932D933C93E1EBF0E0F6
:100370000E94BA160E94DE16A9E9B0E00E940F178B
:1003800083E790E0ADEAB2E08D939C9381E08093A7
:10039000D801ADEAB2E04D915C91A8EDB1E00D91CC
:1003A00011270417150718F011F00C9447050E9447
:1003B000FD11009162000F3F11F40C9400025A925B
:1003C0004A9284E690E0A42DB52D8D939C9382E013
:1003D0000E948A135A924A9281E0A42DB52D8C93E3
:1003E00081E00E948A130E942312249683E00E94D7
:1003F00086130E94D80E8FEF809362000C945401F4
:10040000E1EBF0E0FA93EA930E94DD092296E8E638
:10041000F0E0FA93EA930E949A0922960E94CC0B8C
:100420000091D8010A3311F00C947A030E942C0C2D
:10043000A9E1B1E0EEE3F7E30E943B165A924A923B
:1004400089E1A42DB52D8C9381E00E948A135A92E4
:100450004A9280E0A42DB52D8C9381E00E948A13EE
:10046000E9E1F1E0FA93EA930E944B05269682E0D7
:100470000E948613EEEEF0E00E94BA16E6EDF6E377
:100480000E9420180E94291818F011F00C944A02BA
:100490000C945202AEE0B1E0E2E5F7E30E943B16B5
:1004A0000C946802A8E2B8E0AF93BF93EEEEF0E0E0
:1004B0000E94BA160E94591411E002E0BF91AF9158
:1004C0000E94AF18E8E2F8E0AEE0B1E00E947019D7
:1004D0005A924A9289E1A42DB52D8C9381E00E9415
:1004E0008A135A924A9280E0A42DB52D8C9381E014
:1004F0000E948A13EEE0F1E0FA93EA930E944B0522
:10050000269682E00E948613E6ECF0E00E94BA167E
:10051000EAEDF6E30E9420180E94291810F00C94CE
:10052000D202A8E2B8E0AF93BF93E6ECF0E00E94FD
:10053000BA160E94591411E001E0BF91AF910E94D8
:10054000AF18E8E2F8E0AEE0B1E00E947019E6EC26
:10055000F0E00E94BA16EEEDF6E30E9420180E9429
:10056000291810F00C94D0028CE00E945314EEE095
:10057000F1E0A881B9810E947019AEE0B1E0E8E530
:10058000F7E30E943B16E881F981AEE0B1E00E94FA
:10059000D7130E9470198CE0481A8827580A2296AF
:1005A0000C94D802AEE0B1E0EAE5F7E30E943B1616
:1005B0005A924A9282E3A42DB52D8C9381E00E9439
:1005C0008A135A924A9280E0A42DB52D8C9381E033
:1005D0000E948A13EEE0F1E0FA93EA930E944B0541
:1005E000269682E00E948613A8E2B8E0AF93BF93FC
:1005F000EAEEF0E00E94BA160E94591411E001E000
:10060000BF91AF910E94AF18E8E2F8E0AEE0B1E030
:100610000E947019EAEEF0E00E94BA16E2EEF6E3EC
:100620000E9420180E94291810F00C9433038CE0CB
:100630000E945314EEE0F1E0A881B9810E94701984
:10064000AEE0B1E0E8E5F7E30E943B16E881F9810E
:10065000AEE0B1E00E94D7130E9470198CE0481AF6
:100660008827580A2296EAEEF0E00E94BA16E6EED3
:10067000F6E30E9420180E94291810F00C945C03E5
:100680008CE00E945314EEE0F1E0A881B9810E9451
:100690007019AEE0B1E0E8E5F7E30E943B16E881AF
:1006A000F981AEE0B1E00E94D7130E9470198CE08E
:1006B000481A8827580A22965A924A9280E5A42D11
:1006C000B52D8C9381E00E948A135A924A9280E061
:1006D000A42DB52D8C9381E00E948A13EEE0F1E009
:1006E000FA93EA930E944B05269682E00E948613B5
:1006F0000C947C030E94330E0091D80141E0041B4E
:10070000AAE0B1E00C93AAE0B1E08C91855F8C93F4
:1007100081E08093D4010091D401003318F011F0EE
:100720000C94AA030091D40147E0040FACE0B1E0BF
:100730000C93AAE0B1E04C91ACE0B1E05C9190E0A8
:100740000E94C015A4EDB1E08C918F5F8C9311F0E5
:100750000C948B0381E080930C0100910C01013318
:1007600018F011F00C94D803EEEEF0E00E94BA16E7
:10077000ECE0F1E0A190BB24E5EEF1E0AA0CBB1C9B
:10078000AA0CBB1CEA0DFB1D0E94BF160E94291873
:1007900018F011F00C94CE030C94D0030C94D803F1
:1007A000ACE0B1E08C918F5F8C9311F00C94AD03B1
:1007B000ACE0B1E08C91895F8C9380910C01A8ED45
:1007C000B1E0AD90BB24ACE5B1E0AA0DBB1D8C93AC
:1007D000AAE0B1E04C91A8EDB1E0AD90BB24ACE54E
:1007E000B1E0AA0DBB1D5C9191E00E94C015009183
:1007F000D801013018F011F00C9400040C94150588
:10080000A8EDB1E00D91112741E050E0041B150B5C
:10081000A2EDB1E00D931C93A2EDB1E0AD90BC90C0
:10082000ACE5B1E0AA0DBB1D0D911127A8EDB1E01B
:10083000AD90BB24ACE5B1E0AA0DBB1D4D91552791
:10084000041B150BA0EDB1E00D931C93A0EDB1E0DE
:100850000D911C91003050E015071CF011F00C9424
:1008600033040C943A048091D70180688093D701B7
:100870000C943F048091D7018F778093D701A0ED2E
:10088000B1E08D919C910E94B713A0EDB1E08D93E2
:100890009C93A0EDB1E00D911C91003050E0150744
:1008A0001CF011F00C9456040C941505A0EDB1E069
:1008B0000D911C9142E050E00E949713A2EDB1E02F
:1008C0004D935C93A0EDB1E00D911C91A2EDB1E0D0
:1008D0004D915C91041B150BA0EDB1E00D931C93A1
:1008E0008091D2018093D601A8EDB1E00D9111273E
:1008F00041E050E0041B150BA2EDB1E00D931C93F9
:10090000A2EDB1E0AD90BC90ACE5B1E0AA0DBB1D8D
:100910008C918093D501AAE0B1E08C9181508C93A9
:100920000091D601003018F011F00C9499040C9449
:10093000CE0481E08093D4014091D6010091D4018E
:10094000041718F011F00C94CE040027A7EDB1E0C5
:100950008C9187FB0EF401E041E0041711F00C9438
:10096000B804A5EDB1E08C9181508C930C94BD043A
:10097000A5EDB1E08C918F5F8C93AAE0B1E04C9132
:10098000A5EDB1E05C9191E00E94C015A4EDB1E04D
:100990008C918F5F8C9311F00C949C04AAE0B1E0D1
:1009A0008C918F5F8C938091D0018093D6010091C0
:1009B000D601003018F011F00C94E0040C941505E9
:1009C00081E08093D4014091D6010091D4010417B5
:1009D00018F011F00C9415050027A7EDB1E08C91EB
:1009E00087FB0EF401E041E0041711F00C94FF04C2
:1009F000A5EDB1E08C9181508C930C940405A5ED8C
:100A0000B1E08C918F5F8C93AAE0B1E04C91A5EDA1
:100A1000B1E05C9191E00E94C015A4EDB1E08C9131
:100A20008F5F8C9311F00C94E3040027A7EDB1E0E5
:100A30008C9185FB0EF401E040E0041711F00C945A
:100A40003F05E5E9F0E00E94BF16E9E9F0E00E9409
:100A5000BA160E94C517FF27EDE0A9E9B0E00E9491
:100A60007519E9E9F0E00E943D1BFF27EDE00E94C7
:100A70007C16A1EBB0E0EDE0FF270E947519A8ED10
:100A8000B1E08C918F5F8C9311F00C94C9010C94A0
:100A90005401F894FFCF81E00E94531481E00E943A
:100AA000531482E00E94531481E00E94531481E0A9
:100AB0000E94531481E00E94531481E00E94531459
:100AC00081E00E945314A889B9890E94A619AC85B7
:100AD000BD858C9381E0AE85BF858C93AC85BD854B
:100AE0004C91AE85BF850C91041718F011F00C9451
:100AF0001006AE85BF858C91E889F98901E00A93DB
:100B0000AB85BC850E947B19AEE2B1E0EA85FB852E
:100B1000222791E00E945116A885B9850C93A885DB
:100B2000B9850C91003011F00C949A0581E0A885EC
:100B3000B9858C93A885B9858C9181508C93A885B3
:100B4000B9850C9145E0049FAE81BF810C9280E095
:100B50008093060100910601043018F011F00C9406
:100B60000806E8E1F6E2AE81BF818C919927A8855D
:100B7000B9850E94511880E1AA81BB818C9380E0E5
:100B80008093070100910701043018F011F00C94D4
:100B9000F605A885B9850C91AA81BB814C910423E7
:100BA000AC81BD810C93AA89BB890C91409107014E
:100BB000040FA881B9810C93AC89BD894C91A8819F
:100BC000B9815C91AC81BD819C910E94C015AA81C4
:100BD000BB810C9142E00E9496190C93A7E0B1E012
:100BE0008C918F5F8C9311F00C94C205AC89BD89F8
:100BF0008C918F5F8C93AE81BF818C918F5F8C9332
:100C0000A6E0B1E08C918F5F8C9311F00C94AA0553
:100C1000AE85BF858C918F5F8C9311F00C946E051F
:100C200089E0481A8827580A609608958AE08A93CE
:100C300087E08A938EE78A9387E08A938FEF8A937F
:100C40000E94DC158EE78A9387E08A938EE78A9369
:100C500089E38A938FEF8A930E94DC158EE78A934B
:100C600089E38A938AE08A9389E38A938FEF8A9350
:100C70000E94DC158AE08A9389E38A938AE08A934A
:100C800087E08A938FEF8A930E94DC1549E058E051
:100C900091E00E94C01549E056E191E00E94C01524
:100CA00049E050E291E00E94C01549E055E291E030
:100CB0000E94C01549E05AE291E00E94C01549E047
:100CC00053E391E00E94C01549E058E391E00E948F
:100CD000C0154BE05AE391E00E94C01548E25AE388
:100CE00091E00E94C01544E45AE391E00E94C015CF
:100CF00041E65AE391E00E94C0154DE75AE391E0C6
:100D00000E94C0154FE758E091E00E94C0154FE7E0
:100D100056E191E00E94C0154FE750E291E00E9439
:100D2000C0154FE755E291E00E94C0154FE75AE227
:100D300091E00E94C0154FE753E391E00E94C01577
:100D40004FE758E391E00E94C0154BE056E091E078
:100D50000E94C01548E256E091E00E94C01544E4AC
:100D600056E091E00E94C01541E656E091E00E94F5
:100D7000C0154DE756E091E00E94C0150895A5E822
:100D8000B0E00D911D912D913C9142E050E060E06A
:100D900070E00E94E713ADE9B0E04D935D936D9371
:100DA0007D93A1E8B0E00D911D912D913C91ADE9AD
:100DB000B0E04D915D916D917C910E94FC18ADE881
:100DC000B0E00D931D932D933D93A5E8B0E00D91F8
:100DD0001D912D913C9144E150E060E070E00E9453
:100DE000E713A1E9B0E04D935D936D937D930027E8
:100DF000A7EDB1E08C9185FB0EF401E040E0041713
:100E000011F00C942D07ADE8B0E00D911D912D91DE
:100E10003C914AE050E060E070E00E94E713ADE8EA
:100E2000B0E04D935D936D937D93A9E1B1E0EDE862
:100E3000F0E00E941719E9E1F1E0A8E2B8E00E94B1
:100E40007019E8E2F8E0AEE0B1E01127222704E0F3
:100E500032E00E9464180C943307AEE0B1E0E0E6A3
:100E6000F7E30E943B165A924A9280E0A42DB52DDA
:100E70008C9381E00E948A135A924A928BE3A42DAC
:100E8000B52D8C9381E00E948A13EEE0F1E0FA9395
:100E9000EA930E944B05269682E00E948613002763
:100EA000A7EDB1E08C9185FB0EF401E040E0041762
:100EB00011F00C947107ADE8B0E00D911D912D91EA
:100EC0003C91A1E9B0E04D915D916D917C910E94C2
:100ED000F718ADE8B0E00D931D932D933D930C945E
:100EE0008307A1E8B0E00D911D912D913C914AE05E
:100EF00050E060E070E00E94E713ADE8B0E04D9391
:100F00005D936D937D93A9E1B1E0EDE8F0E00E947F
:100F10001719E9E1F1E0A8E2B8E00E947019E8E2EF
:100F2000F8E0AEE0B1E01127222704E032E00E94B1
:100F300064185A924A9288E3A42DB52D8C9381E0CF
:100F40000E948A135A924A928BE3A42DB52D8C935A
:100F500081E00E948A13EEE0F1E0FA93EA930E94A6
:100F60004B05269682E00E9486130027A7EDB1E08C
:100F70008C9185FB0EF401E040E0041711F00C9415
:100F8000ED07ADE8B0E00D911D912D913C91A1E9E7
:100F9000B0E04D915D916D917C910E94F718ADE8A4
:100FA000B0E00D931D932D933D93A9E1B1E0EDE8E1
:100FB000F0E00E941719E9E1F1E0A8E2B8E00E9430
:100FC0007019E8E2F8E0AEE0B1E01127222704E072
:100FD00032E00E9464180C94F307AEE0B1E0E0E662
:100FE000F7E30E943B165A924A9286E6A42DB52D4D
:100FF0008C9381E00E948A135A924A928BE3A42D2B
:10100000B52D8C9381E00E948A13EEE0F1E0FA9313
:10101000EA930E944B05269682E00E948613A9E17E
:10102000B1E0E6E6F7E30E943B165A924A9283E06B
:10103000A42DB52D8C9381E00E948A135A924A9276
:1010400083E2A42DB52D8C9381E00E948A13E9E1FF
:10105000F1E0FA93EA930E944B05269682E00E9403
:101060008613A9E1B1E0E8E6F7E30E943B165A9245
:101070004A9283E0A42DB52D8C9381E00E948A13BF
:101080005A924A9288E2A42DB52D8C9381E00E9459
:101090008A13E9E1F1E0FA93EA930E944B05269660
:1010A00082E00E948613A9E1B1E0EAE6F7E30E943C
:1010B0003B165A924A9283E0A42DB52D8C9381E081
:1010C0000E948A135A924A9281E3A42DB52D8C93E3
:1010D00081E00E948A13E9E1F1E0FA93EA930E9429
:1010E0004B05269682E00E948613A9E1B1E0ECE66A
:1010F000F7E30E943B165A924A9280E0A42DB52D48
:101100008C9381E00E948A135A924A9286E0A42D21
:10111000B52D8C9381E00E948A13E9E1F1E0FA9306
:10112000EA930E944B05269682E00E948613A9E16D
:10113000B1E0EEE6F7E30E943B165A924A9280E055
:10114000A42DB52D8C9381E00E948A135A924A9265
:1011500084E1A42DB52D8C9381E00E948A13E9E1EE
:10116000F1E0FA93EA930E944B05269682E00E94F2
:101170008613A9E1B1E0E0E7F7E30E943B165A923B
:101180004A9280E0A42DB52D8C9381E00E948A13B1
:101190005A924A928EE1A42DB52D8C9381E00E9443
:1011A0008A13E9E1F1E0FA93EA930E944B0526964F
:1011B00082E00E948613A9E1B1E0E2E7F7E30E9432
:1011C0003B165A924A9280E0A42DB52D8C9381E073
:1011D0000E948A135A924A9285E3A42DB52D8C93CE
:1011E00081E00E948A13E9E1F1E0FA93EA930E9418
:1011F0004B05269682E00E948613E9EAF0E0A9E119
:10120000B1E00E9470195A924A9280E0A42DB52D47
:101210008C9381E00E948A135A924A9280E0A42D16
:10122000B52D8C9381E00E948A13E9E1F1E0FA93F5
:10123000EA930E944B05269682E00E948613089549
:101240000E94AD150E94BA15E1E0F0E00E94DE13A5
:101250008CE90E94A415A9E1B1E0E4E7F7E30E945C
:101260003B165A924A928DE1A42DB52D8C9381E0C4
:101270000E948A135A924A9284E1A42DB52D8C9330
:1012800081E00E948A13E9E1F1E0FA93EA930E9477
:101290004B05269682E00E948613A9E1B1E0E4E8BE
:1012A000F7E30E943B165A924A9289E1A42DB52D8C
:1012B0008C9381E00E948A135A924A928EE1A42D67
:1012C000B52D8C9381E00E948A13E9E1F1E0FA9355
:1012D000EA930E944B05269682E00E948613A9E1BC
:1012E000B1E0E6E9F7E30E943B165A924A9288E39E
:1012F000A42DB52D8C9381E00E948A135A924A92B4
:1013000082E3A42DB52D8C9381E00E948A13E9E13C
:10131000F1E0FA93EA930E944B05269682E00E9440
:101320008613E2E0F0E00E94DE130E94AD150E94F9
:10133000BA1508958C9A8D9A9598A881B98190E2F2
:101340008D91983018F4392F992702C038E09850C1
:101350008795949808F4949A00000000959A0000EC
:1013600000009598000000003A9591F7992341F705
:1013700081E080936C008C9A8D9A9598ACE6B0E0F1
:1013800098E08D91983018F4392F992702C038E0F1
:1013900098508795949808F4949A00000000959AC4
:1013A000000000009598000000003A9591F79923FD
:1013B00041F7969A000096980895A881B9810D91F9
:1013C0001D912D913C91A5EBB0E00D931D932D93B4
:1013D0003C9380E197E2ADEBB0E08D939C9300E00D
:1013E00010E020E030E0A8E6B0E00D931D932D93CF
:1013F0003C93A5EBB0E00D911C91ADEBB0E04D91AD
:101400005C910E94BD13A9EBB0E04D935C9381E029
:1014100090E0ABEBB0E08D939C93A9EBB0E04D91E5
:101420005C91ABEBB0E00D911C910417150718F01F
:1014300011F00C94480AA8E6B0E00D911D912D9191
:101440003C91ADE6B0E04D915D916D917C910E9433
:10145000F718A8E6B0E00D931D932D933D93A5EBEF
:10146000B0E00D911D912D913C9140E157E260E07B
:1014700070E00E94FC18A5EBB0E00D931D932D9336
:101480003D93ABEBB0E00E948E1311F00C940D0A6B
:1014900088EE93E0ADEBB0E08D939C93A5EBB0E0CC
:1014A0000D911C91ADEBB0E04D915C910E94BD138C
:1014B000A9EBB0E04D935C9381E090E0ABEBB0E042
:1014C0008D939C93A9EBB0E04D915C91ABEBB0E0B8
:1014D0000D911C910417150718F011F00C949D0A3A
:1014E000A8E6B0E00D911D912D913C91A1E7B0E0EF
:1014F0004D915D916D917C910E94F718A8E6B0E046
:101500000D931D932D933D93A5EBB0E00D911D918F
:101510002D913C9148EE53E060E070E00E94FC1891
:10152000A5EBB0E00D931D932D933D93ABEBB0E095
:101530000E948E1311F00C94620A84E690E0ADEBE9
:10154000B0E08D939C93A5EBB0E00D911C91ADEBB9
:10155000B0E04D915C910E94BD13A9EBB0E04D93BA
:101560005C9381E090E0ABEBB0E08D939C93A9EBB2
:10157000B0E04D915C91ABEBB0E00D911C91041784
:10158000150718F011F00C94F20AA8E6B0E00D91DE
:101590001D912D913C91A5E7B0E04D915D916D912C
:1015A0007C910E94F718A8E6B0E00D931D932D934F
:1015B0003D93A5EBB0E00D911D912D913C9144E63A
:1015C00050E060E070E00E94FC18A5EBB0E00D93E5
:1015D0001D932D933D93ABEBB0E00E948E1311F061
:1015E0000C94B70A8AE090E0ADEBB0E08D939C9349
:1015F000A5EBB0E00D911C91ADEBB0E04D915C918D
:101600000E94BD13A9EBB0E04D935C9381E090E0A4
:10161000ABEBB0E08D939C93A9EBB0E04D915C9166
:10162000ABEBB0E00D911C910417150718F011F009
:101630000C94470BA8E6B0E00D911D912D913C91C3
:10164000A9E7B0E04D915D916D917C910E94F718F2
:10165000A8E6B0E00D931D932D933D93A5EBB0E06C
:101660000D911D912D913C914AE050E060E070E0B9
:101670000E94FC18A5EBB0E00D931D932D933D93B4
:10168000ABEBB0E00E948E1311F00C940C0BA5EBA9
:10169000B0E08D919C91A9EBB0E08D939C9381E09B
:1016A00090E0ABEBB0E08D939C93A9EBB0E04D9153
:1016B0005C91ABEBB0E00D911C910417150718F08D
:1016C00011F00C947E0BA8E6B0E00D911D912D91C8
:1016D0003C91ADE7B0E04D915D916D917C910E94A0
:1016E000F718A8E6B0E00D931D932D933D93ABEB57
:1016F000B0E00E948E1311F00C94550B089500E099
:1017000010E020E030E0A8E6B0E00D931D932D93AB
:101710003C938C9A8D9A9598A8E6B0E090E28D91D2
:10172000983018F4392F992702C038E098508795DF
:10173000949808F4949A00000000959A0000000024
:101740009598000000003A9591F7992341F780E0C1
:1017500080936C008C9A8D9A9598ACE6B0E098E0F6
:101760008D91983018F4392F992702C038E098509D
:101770008795949808F4949A00000000959A0000C8
:1017800000009598000000003A9591F7992341F7E1
:10179000969A00009698089580E090E0AFEBB0E054
:1017A0008D939C9380E090E0A1ECB0E08D939C93AE
:1017B00080E092E0A3ECB0E08D939C939798A3EC2B
:1017C000B0E00D911C91003050E0150718F011F0B9
:1017D0000C94EC0B0C94290CA8980027BB27A3E3CE
:1017E0008C9181FB0EF401E041E0041711F00C94A0
:1017F000070CAFEBB0E00D911C91A3ECB0E04D9164
:101800005C91040F151FAFEBB0E00D931C93002704
:10181000BB27A3E38C9182FB0EF401E041E00417A7
:1018200011F00C94210CA1ECB0E00D911C91A3ECF3
:10183000B0E04D915C91040F151FA1ECB0E00D9349
:101840001C93A89A91E0A3ECB0E00E9441160C947E
:10185000DF0B979AA89A0895EAEEF6E30E94201803
:10186000E1ECF0E0D190E080FF2400270E94DE163A
:101870000E948517FF27EDE0A6ECB0E00E947519E5
:10188000EEEEF6E30E942018E6ECF0E00E94BA16B5
:101890000E94B617FF27EDE0A6ECB0E00E94751994
:1018A000E2EFF6E30E942018EFEBF0E0D190E08049
:1018B000FF2400270E94DE160E948517FF27EDE017
:1018C000AAECB0E00E947519E6EFF6E30E9420183A
:1018D000E6ECF0E00E94BA160E942F17FF27EDE019
:1018E000AAEFB0E00E947519AEEFB0E0EAEFF6E3C0
:1018F0000E947F13EEEFF0E0AAEFB0E00E94001B21
:10190000FF27EDE0AEECB0E00E947519EEECF0E0E0
:101910000E94BF16EEEFF6E30E9417180E942F17E1
:10192000FF27EDE0AEECB0E00E947519EEECF0E0C0
:101930000E94BF16EEEFF6E30E9417180E94C5172B
:10194000FF27EDE0AAEFB0E00E947519EEECF0E0A1
:101950000E94BF16EEEFF6E30E9417180E94B6171A
:10196000FF27EDE0AEEFB0E00E947519EEEFF0E07A
:101970000E94BF16EAEFF0E00E94BA160E942F17ED
:10198000FF27EDE0A2E0B1E00E947519E2E0F1E08E
:101990000E94AC19FF27EDE0AEEEB0E00E94751991
:1019A000E2E0F7E30E942018EAECF0E00E94BA16A9
:1019B0000E942F17FF27EDE0AAEFB0E00E947519F3
:1019C000EAEFF0E00E94CB19FF27EDE0A2EDB0E0D6
:1019D0000E947519EAEFF0E00E94221BFF27EDE05C
:1019E000A6EDB0E00E947519EEECF0E00E94BF1683
:1019F000E2EDF0E00E94BA160E948517FF27EDE0A5
:101A0000AAEDB0E00E947519EEECF0E00E94BF165E
:101A1000E6EDF0E00E94BA160E948517FF27EDE080
:101A2000AEEDB0E00E947519EAEDF0E00E94BF163D
:101A3000EEEFF6E30E9417180E94B617FF27EDE0BD
:101A4000AAEFB0E00E947519EAEFF0E00E94BF161D
:101A5000EAEFF0E00E94BA160E948517FF27EDE03A
:101A6000A2EFB0E00E947519EEEDF0E00E94BF1603
:101A7000EEEDF0E00E94BA160E948517FF27EDE018
:101A8000A6EFB0E00E947519E6EFF0E00E94BF16E5
:101A9000E2EFF0E00E94BA160E94C517FF27EDE0C2
:101AA000AAEFB0E00E947519EEEDF0E00E94BF16BB
:101AB000E6E0F7E30E9417180E948517FF27EDE084
:101AC000AEEFB0E00E947519EAEFF0E00E94BF1699
:101AD000EEEFF0E00E94BA160E942F17FF27EDE00C
:101AE000A2E0B1E00E947519EAE0F7E30E94201835
:101AF000E2E0F1E00E94BA160E948517FF27EDE0B0
:101B0000AAEFB0E00E947519EAEFF0E00E94AC196C
:101B1000FF27EDE0A2EEB0E00E947519EAEDF0E0DB
:101B20000E94BF16EAEDF0E00E94BA160E948517E7
:101B3000FF27EDE0AAEFB0E00E947519EAEFF0E0B0
:101B40000E94BF16EEEFF6E30E9417180E94B61728
:101B5000FF27EDE0AEEFB0E00E947519E6EFF0E090
:101B60000E94BF16EEEFF0E00E94BA160E94B61770
:101B7000FF27EDE0AAEFB0E00E947519E6EFF0E074
:101B80000E94BF16E2EFF0E00E94BA160E94C5174D
:101B9000FF27EDE0AEEFB0E00E947519EEEFF0E048
:101BA0000E94BF16EAEFF0E00E94BA160E942F17BB
:101BB000FF27EDE0A2E0B1E00E947519EAE0F7E34B
:101BC0000E942018E2E0F1E00E94BA160E948517F8
:101BD000FF27EDE0AAEFB0E00E947519EAEFF0E010
:101BE0000E94AC19FF27EDE0A6EEB0E00E94751947
:101BF000E6EEF0E00E94BF16E6EEF0E00E94BA16B4
:101C00000E948517FF27EDE0AAEFB0E00E9475194A
:101C1000E2EEF0E00E94BF16E2EEF0E00E94BA169B
:101C20000E948517FF27EDE0AEEFB0E00E94751926
:101C3000EEEFF0E00E94BF16EAEFF0E00E94BA1665
:101C40000E94C517FF27EDE0A2E0B1E00E947519E0
:101C5000E2E0F1E00E94471BFF27EDE0AAEEB0E0D2
:101C60000E9475190895EAEEF6E30E942018E1EC4F
:101C7000F0E0D190E080FF2400270E94DE160E9451
:101C80008517FF27EDE0A6ECB0E00E947519EEEE97
:101C9000F6E30E942018E6ECF0E00E94BA160E94DB
:101CA000B617FF27EDE0A6ECB0E00E947519E2EF51
:101CB000F6E30E942018EFEBF0E0D190E080FF24E3
:101CC00000270E94DE160E948517FF27EDE0AAEC90
:101CD000B0E00E947519E6EFF6E30E942018E6ECEA
:101CE000F0E00E94BA160E942F17FF27EDE0AAEF3E
:101CF000B0E00E947519AEEFB0E0EAEFF6E30E94A3
:101D00007F13EEEFF0E0AAEFB0E00E94001BFF2788
:101D1000EDE0AEECB0E00E947519EEECF0E00E9450
:101D2000BF16EEEFF6E30E9417180E942F17FF2749
:101D3000EDE0AEECB0E00E947519EEECF0E00E9430
:101D4000BF16EEEFF6E30E9417180E94C517FF2793
:101D5000EDE0AAEFB0E00E947519EEECF0E00E9411
:101D6000BF16EEEFF6E30E9417180E94B617FF2782
:101D7000EDE0AEEFB0E00E947519EEEFF0E00E94EA
:101D8000BF16EAEFF0E00E94BA160E942F17FF2755
:101D9000EDE0A2E0B1E00E947519E2E0F1E00E94FE
:101DA000AC19FF27EDE0AEEEB0E00E947519089582
:101DB000009162000D3F11F00C945A0FA5E8B0E0BD
:101DC0000D911D912D913C9142E050E060E070E05A
:101DD0000E94E713ADE9B0E04D935D936D937D9361
:101DE000A1E8B0E00D911D912D913C91ADE9B0E0DD
:101DF0004D915D916D917C910E94F718ADE9B0E035
:101E00000D931D932D933D93ADE9B0E00D911D9180
:101E10002D913C91A9E8B0E04D915D916D917C913F
:101E20000E94F718ADE9B0E00D931D932D933D93FB
:101E300040E65AEE60E070E0ADE9B0E00D911D9132
:101E40002D913C910E9401191CF011F00C942A0F65
:101E50000C94460F5A924A9282E390E0A42DB52D3D
:101E60008D939C9382E00E948A135A924A9282E058
:101E7000A42DB52D8C9381E00E948A130E94231219
:101E8000249683E00E9486130C945A0FA1E8B0E0D8
:101E90000D911D912D913C91A9E8B0E04D915D917E
:101EA0006D917C910E94F718A1E8B0E00D931D930D
:101EB0002D933D93009162000E3F11F00C94DA0FC8
:101EC000A5E8B0E00D911D912D913C9142E050E0CC
:101ED00060E070E00E94E713ADE9B0E04D935D93E0
:101EE0006D937D93A1E8B0E00D911D912D913C91F2
:101EF000ADE9B0E04D915D916D917C910E94FC182F
:101F0000ADE9B0E00D931D932D933D93ADE9B0E0A5
:101F10000D911D912D913C91A9E8B0E04D915D91FD
:101F20006D917C910E94FC18ADE9B0E00D931D937A
:101F30002D933D9348EE53E060E070E0ADE9B0E0F2
:101F40000D911D912D913C910E9401190CF402C03C
:101F50000C94C60F5A924A9282E390E0A42DB52DBC
:101F60008D939C9382E00E948A135A924A9282E057
:101F7000A42DB52D8C9381E00E948A130E94231218
:101F8000249683E00E9486130C94DA0FA1E8B0E057
:101F90000D911D912D913C91A9E8B0E04D915D917D
:101FA0006D917C910E94FC18A1E8B0E00D931D9307
:101FB0002D933D9300916200073F11F00C94B610F1
:101FC0008091D7018F7D8093D7010091AF000A30B7
:101FD00011F00C9407105A924A9282E390E0A42DDB
:101FE000B52D8D939C9382E00E948A135A924A9257
:101FF00082E0A42DB52D8C9381E00E948A130E946B
:102000002312249683E00E9486130C94B61000914C
:10201000AF0041E0040FA0EBB0E00C93ECEEF5E272
:10202000A0EBB0E08C919927A5EAB0E00E9454188B
:10203000A5EAB0E00D911D912D913C9142E050E058
:1020400060E070E00E94E713ADE9B0E04D935D936E
:102050006D937D93A1E8B0E00D911D912D913C9180
:10206000ADE9B0E04D915D916D917C910E94FC18BD
:10207000ADE9B0E00D931D932D933D93A5EAB0E03B
:102080000D911D912D913C9142E050E060E070E097
:102090000E94E713A1EAB0E04D935D936D937D93A9
:1020A000A1E8B0E00D911D912D913C91A1EAB0E025
:1020B0004D915D916D917C910E94F718A1EAB0E07D
:1020C0000D931D932D933D9348EE53E060E070E037
:1020D000ADE9B0E00D911D912D913C910E94011947
:1020E00080E00CF481E08F9340E65AEE60E070E00F
:1020F000A1EAB0E00D911D912D913C910E94011932
:1021000080E014F009F081E09F91892B882311F47D
:102110000C94A6105A924A9282E390E0A42DB52D19
:102120008D939C9382E00E948A135A924A9282E095
:10213000A42DB52D8C9381E00E948A130E94231256
:10214000249683E00E9486130C94B6108091B00010
:102150008093AF00A5EAB0E00D911D912D913C91C7
:10216000A5E8B0E00D931D932D933C930091620080
:102170000B3F11F00C9478110091AF00003011F07A
:102180000C94C9108091D70180628093D7010C9480
:1021900078110091AF0041E0041BA0EBB0E00C937C
:1021A000ECEEF5E2A0EBB0E08C919927A5EAB0E067
:1021B0000E945418A5EAB0E00D911D912D913C911B
:1021C00042E050E060E070E00E94E713ADE9B0E06B
:1021D0004D935D936D937D93A1E8B0E00D911D91BA
:1021E0002D913C91ADE9B0E04D915D916D917C9167
:1021F0000E94FC18ADE9B0E00D931D932D933D9323
:10220000A5EAB0E00D911D912D913C9142E050E086
:1022100060E070E00E94E713A1EAB0E04D935D93A7
:102220006D937D93A1E8B0E00D911D912D913C91AE
:10223000A1EAB0E04D915D916D917C910E94F718FB
:10224000A1EAB0E00D931D932D933D9348EE53E02A
:1022500060E070E0ADE9B0E00D911D912D913C91F1
:102260000E94011980E00CF481E08F9340E65AEE61
:1022700060E070E0A1EAB0E00D911D912D913C91DC
:102280000E94011980E014F009F081E09F91892BF0
:10229000882311F40C9468115A924A9282E390E0D8
:1022A000A42DB52D8D939C9382E00E948A135A929F
:1022B0004A9282E0A42DB52D8C9381E00E948A136E
:1022C0000E942312249683E00E9486130C947811B6
:1022D0008091B0008093AF00A5EAB0E00D911D9110
:1022E0002D913C91A5E8B0E00D931D932D933C9367
:1022F000009162000F3D11F00C94BA110091AE00F4
:10230000093011F00C94A0115A924A9282E390E0A5
:10231000A42DB52D8D939C9382E00E948A135A922E
:102320004A9282E0A42DB52D8C9381E00E948A13FD
:102330000E942312249683E00E9486130C94BA1103
:10234000AEEAB0E08C918F5F8C93E2E9F5E2AEEA01
:10235000B0E08C919927A9E8B0E00E945418EAEB0C
:10236000F5E2AEEAB0E08C910E945B18A9EAB0E019
:102370000E943B16009162000F3E11F00C94FC117C
:102380000091AE00003011F00C94E2115A924A9282
:1023900082E390E0A42DB52D8D939C9382E00E9462
:1023A0008A135A924A9282E0A42DB52D8C9381E033
:1023B0000E948A130E942312249683E00E948613AF
:1023C0000C94FC11AEEAB0E08C9181508C93E2E960
:1023D000F5E2AEEAB0E08C919927A9E8B0E00E945E
:1023E0005418EAEBF5E2AEEAB0E08C910E945B187B
:1023F000A9EAB0E00E943B160895A1E6B0E089B3D7
:102400008C93009161000F3F11F40C942212809183
:1024100061008093620089E190E00E94441480E0B2
:1024200080936100009161000F3F11F40C941E1223
:10243000A1E6B0E089B38C930C94121289E190E08C
:102440000E944414089581E090E0A3E6B0E08D93EB
:102450009C93AA81BB814D915C91A3E6B0E00D9164
:102460001C910417150718F011F00C946412BB2787
:10247000A2E38C9181FB882780F9809580FBBB27A4
:10248000A2E38C9181F98C93A881B9818C919927D1
:102490000E944414BB27A2E38C9181FB882780F91A
:1024A000809580FBBB27A2E38C9181F98C93A88156
:1024B000B9818C9199270E944414A3E6B0E00E9450
:1024C0008E1311F00C9429120895F894FFCF588AB6
:1024D0006042158C0E427502B841D8F07641C44274
:1024E0003041C18B07417F6ADF40D786C140C2516E
:1024F000AC4005179B4086C98B40D39F7B404278F8
:10250000624083A34C40F4893A40C53D2C40E674B8
:102510002140B79C194098FA1340E6CB0F404E6219
:102520000C40A835094029ED0540B35E0240A110DA
:10253000FD3F7906F53F3EEDEC3F3815E53F5EBACD
:10254000DD3F38F8D63F8AC8D03F9E07CB3F518346
:10255000C53F1B0DC03FC68ABA3F8104B53F8BA65D
:10256000AF3FAEB6AA3F077CA63FB116A33F8F533D
:10257000A03F5A819D3F9560993F4547923FCDCC02
:102580008C3F6666863F0AD7833FAE47813F000097
:10259000803F0A00000014000000320000006400C8
:1025A0000000C8000000F4010000E8030000D007AC
:1025B000000088130000102700002031304B00205D
:1025C00032304B002035304B003130304B00323050
:1025D000304B003530304B002020314D0020203270
:1025E0004D002020354D002031304D0014000000FA
:1025F0003200000064000000C8000000F401000088
:10260000E8030000D0070000881300001027000036
:10261000204E000050C300000008101508000304FD
:10262000081000081F1F0800021F1F020000000002
:10263000000000010000000004040400000B150964
:1026400000001D15120000101718000E11110E00C9
:10265000091F0100000B151509000A11150E0006CF
:102660000A1F02001D15151200020D15020010139D
:102670001418000A15150A000815160C000F14147A
:102680000F001F15150A000E111111001F11110E58
:10269000001F151111001F141010000E1115170046
:1026A0001F04041F00111F1100001211111E001F32
:1026B000040A11001F010101001F18181F001F1834
:1026C000061F000E11110E001F141408000E111326
:1026D0000F001F141609000915151200101F100015
:1026E000001E01011E001C02011E001F03031F002B
:1026F000110A061900110A0418001315151984E0AF
:10270000C89531960D928A95D9F70895481A882769
:10271000580A0895480E8827581E0895ED91FC9197
:102720003196FC93EE93089500FC10D0089503D0E9
:1027300024D001F8F9CF0024E89457FF02C009D053
:10274000689400F80BD010F80124089502D009D045
:102750000895509540954F5F5F4F0895E89417FF97
:102760000895009510950F5F1F4F68940895992361
:102770001AF48095909501960895352F242FE894AA
:10278000452B11F468940895512F402F00271127ED
:1027900080E1440F551F001F111F021B130B4160E6
:1027A00018F4020F131F4E7F8A9599F708958F939F
:1027B0008D918823E9F711978F91089588EE93E022
:1027C00063D03197D9F7089500FC05D0089530D033
:1027D00005D001F8F9CF37D03FD00895842F952F39
:1027E000A62FB72FE894452B462B472B11F468945E
:1027F0000895402F512F622F732F00271127222772
:102800003327F0E2440F551F661F771F001F111F6B
:10281000221F331F081B190B2A0B3B0B416028F4A6
:10282000080F191F2A1F3B1F4E7FFA9559F708956D
:102830000024E89477FF02C006D0689400F809D01D
:1028400010F80124089512D04F5F5F4F6F4F7F4FF4
:102850000895E89437FF08950095109520953095D8
:102860000F5F1F4F2F4F3F4F68940895409550952D
:102870006095709508953197F1F70895689462F81E
:102880000895E89462F80895EF93FF93EE27E82BFC
:10289000E92B31F0EEE3FDE03197F1F70197D1F745
:1028A000FF91EF9108955A924A92480E8827581E38
:1028B00008958DE207FD8D938F2D881F802F881F2F
:1028C0008F57082F6894F7F8802F87FF15C08095E1
:1028D0008395082F80E38D938EE28D93802F815214
:1028E00028F080E38D9399279C93089544270A95B7
:1028F000802F09F196D01FC0805230F09EE49D9346
:1029000081E48D939D93EFCF4427DF92EF92FF9266
:102910000F938FE1801B11F0082F83D089D09EE2A6
:102920009D930F91FF90EF90DF9044270395003225
:1029300009F4D7CF2BD03F93E2ECF9E238E12F2D09
:102940001E2D0D2DFF24EE24DD244427000F111F22
:10295000221FA8F42F923F920E941318102C0E945D
:102960001318202C0E941318302C0E941318319732
:10297000410DD21CE31CF01C3F902F9001C03396F8
:1029800031963A9519F73F9107D0AFCFDD0CEE1C89
:10299000FF1C0A95D9F70895002719E058D08F93A6
:1029A000802B11F0039501C08F911A95B9F7802FF4
:1029B000882309F496CF8F91805D8D930A95D9F77E
:1029C00092CF0065CD1D80B2E60E40597307A0ACD2
:1029D000B90350D6DC01286BEE0094357700CA9A13
:1029E0003B0065CD1D00B2E60E0059730700ACB97F
:1029F0000300D6DC01006BEE0000357700009A3B47
:102A00000000CD1D0000E60E000073070000B903B2
:102A10000000DC010000EE000000770000003B0039
:102A20000000F694E794D79447950A95D1F7089556
:102A300000270DD08F9303958F2D8E298D29842B00
:102A4000C1F78F91805D8D930A95D9F74CCF1F9375
:102A50000F93002710E2440FDD1CEE1CFF1C001F2B
:102A6000802F9AE0890B10F0082F43951A9599F75B
:102A7000802F0F911F9108952093B1023093B202DD
:102A80004093B3025093B40208952091B102309163
:102A9000B2024091B3025091B4020895AA98AF983F
:102AA000AB9AAC9A84E699270E944414AF9A88277F
:102AB00036D083E034D082E447D080E130D088271C
:102AC0002ED083E441D088272AD029D080E43CD07E
:102AD00080E125D0882723D081E436D080E834D027
:102AE0008FE932D00895AE9A992797BB9FEF98BB94
:102AF000AC9800000000AD9800000000000000004D
:102B00000000000096B300000000AC9A0000000036
:102B1000AD9A9370933061F79FEF97BB0895E3DF11
:102B2000AE9888BB00000000AB9800000000AD9894
:102B3000000000000000000000000000AB9A000050
:102B40000000AD9A00000895CEDFAE9AEACF842F40
:102B5000E6DF852FE4DF84E2F7CF40E053E0F7DFE4
:102B6000E0E0F4E08827DBDFDADF80ECEDDF3197AF
:102B7000C9F7089544275527EADFE0E8F0E0F2CFEF
:102B8000042F48E0D3D30F9307E0081B802F99232D
:102B900011F4877001C08860982F00E1452FBAD3E7
:102BA0008F91480F8827581F40505D4F9F93CFDF6C
:102BB0009F9180EF890FC8CFAA24BB24FF24EC810A
:102BC000EA80EE1AFF08FB81298033242F1A33088C
:102BD00081E0EA14FA043CF42FEF3FEFE094F09424
:102BE000E80EFA1C02C021E033272A143A043CF410
:102BF0006FEF7FEF20943094280E3A1C02C061E002
:102C0000772735D02E143F0414F009F017C0CE2CCE
:102C1000DF2CCC0CDD1C022C132C000C111C9A8117
:102C2000E91761F0E20FA00CB11CAE14BF0424F050
:102C300019F0F60FAC18BD081AD0F1CFC22CD32C66
:102C4000CC0CDD1C0E2C1F2C000C111C9981F917CB
:102C500011F425960895F60FA00CB11CA214B3042C
:102C600024F019F0E20FAC18BD0801D0EFCF4E2FC1
:102C70005F2F988185CF0E9413180D920020D9F7FD
:102C80000895903041F00D911C91169507959A95F5
:102C9000E1F71C930E93089599910027A90FB01F97
:102CA0001197492F4A955E2F6F2FE894112743956E
:102CB000203019F0C895802D01C080818823B9F09B
:102CC0007C917723A1F0781739F40EF0042F139537
:102CD000689411963196EBCF112321F0411BA11B73
:102CE0001127B10BE894E52FF62F1196E0CF88233A
:102CF00011F00027089508953DD0992711278F2DB1
:102D0000880F80E8F82A802F881F08F41FEF41F011
:102D10008F57082F07FD04C0003240F08FEF01C02D
:102D20008827982FD82EE82EF82E09C08FE1801B17
:102D3000082FF694E794D79497950A95D1F7112325
:102D400051F09095D094E094F09481E0980F88270A
:102D5000D81EE81EF81E0F2DFE2CED2CD92E08953E
:102D6000D094E094F09491E0D90E9927E91EF91ED1
:102D700010950895D190E190F190019108952191DD
:102D80003191419151910895102F90E8FF0C001F4F
:102D90000927990FF7941078652F90E8440F551F75
:102DA0005927990F4795607800380895FF0C90E8EF
:102DB0009027110F9795F794092F0895102FBD2C88
:102DC000DE2CEF2CF02E11234AF4B094D094E09432
:102DD000F0949FEFB91AD90AE90AF90A0EE1FF2027
:102DE00039F4FE2CED2CDB2CBB240850C2F76BC051
:102DF00032F00A95BB0CDD1CEE1CFF1CF9CF01D094
:102E0000D5CFB7FE089590E8B91611F4D0FE089515
:102E10009FEFD91AE90AF90A09F403950895DD929A
:102E2000ED92FD920C930895502F2D2D3E2D4F2D98
:102E3000612F08952DEC3CEC4CEC5DE366270FC050
:102E400099DFF2DFDD24EE2490E8F92E0FE307C0CE
:102E500096DF05C02227332740E251E46627552339
:102E600051F1002381F190DF71F11627005850587D
:102E70000894050B18F407FD03C025C007FD23C007
:102E8000469537952795F694E794D79422D0FF205E
:102E90002AF0DD0CEE1CFF1C015073F09D2D969561
:102EA00048F0DD203AF4EE202AF491E0D90E99277B
:102EB000E91EF91E7BCF07C09FE7092FF92A9FEF74
:102EC000D92EE92E0895DD24EE24FF2400271127B2
:102ED00008959F929924AA24BB2488E1D216E30680
:102EE000F40628F0D21AE30AF40A089401C0889480
:102EF000991CAA1CBB1CDD0CEE1CFF1C8A9571F7EB
:102F0000D92CEA2CFB2C9F9008953EDFE1F250383B
:102F1000D1F21627005850580894051F12F418F4DF
:102F2000CBCF08F0D0CF0AD0FF202AF0BB0CDD1C9D
:102F3000EE1CFF1C3BCF0F5FFBF138CF9F92992413
:102F4000AA24BB24992788E1990CAA1CBB1CDD1C70
:102F5000EE1CFF1C30F4920EA31EB41ED91EE91EF7
:102F6000F91E8A9589F79F90089509DF0DDF503883
:102F700029F090E869270CC00AF045D017CF5FE32D
:102F800022273327442701C0FADEFEDE5038B1F392
:102F9000003899F3902F951B8BF312F434D0FACFAD
:102FA000983118F0222733274427983028F0232F10
:102FB000342F44279850F9CF992329F04695379517
:102FC00027959A95D9F7912F962742F014D0B0F60D
:102FD000F794E794D7940F5F8BF66ECF10D051F033
:102FE00008F4BEDEFF2052F2DD0CEE1CFF1C015087
:102FF000CBF762CF68CFD20EE31EF41E0895D21A2B
:10300000E30AF40A0895DF92EF92FF920F931F9361
:10301000D22EE32EF42E052F162F6F915F914F9134
:103020003F912F910895C895319600200895FBDFB8
:10303000D02CF9DFE02CF7DFF02CF5DF002D089520
:10304000F2DF202DF0DF302DEEDF402DECDF502DB4
:10305000089507FB00680EF40F7757FB50680EF4D5
:103060005F7707FD02C057FF05C0D216E306F406DE
:10307000050708952D153E054F05500708950024B6
:103080000D280E280F28002A0020089581E003C093
:1030900082E001C084E0C8950D9231968A95D9F7F7
:1030A0000895E80FF91FF2CF880F991F880F991F15
:1030B000E80FF91FEFCF882331F0C8953196002033
:1030C000E1F78A95D1F708952E2E3F2E9927819109
:1030D0008D3209F093958823D1F79A95E22DF32D3F
:1030E000112361F0091718F011F0101B01C0191B12
:1030F00028F021F080E28D931A95E9F780818D32D6
:1031000019F48D93319604C0222311F08BE28D9334
:10311000091738F031F0091B21F080E38D930A95EF
:10312000E9F781918D938823E1F7332351F0EA2F5A
:10313000FB2F319633958E9182933A95E1F78EE28B
:103140008C93089599278D9193958823E1F7939512
:1031500011968C9311978E919A95D1F70895EA2F35
:10316000FB2F00244C918D9103948E32E1F71124B2
:103170008D9113948823E1F71A94101640F4119757
:10318000202F2119239580E38D932A95E9F711309B
:1031900039F59927AE2FBF2FA00DB91FA00FB91F6A
:1031A0008C919C93853308F421C031E08E918E324E
:1031B000E9F38D3241F0830F8A3319F480E331E073
:1031C00001C033278C93AE1789F7332341F0AE2F1C
:1031D000BF2FB8DF81E34D3209F431968083089523
:1031E0008827E00DF81FE00FF81F80830895040F73
:1031F000151F261F371F0895041B150B260B370BB1
:10320000089504171507260737070895000F111FA3
:10321000221F331F089500951095209530950F5F5C
:103220001F4F2F4F3F4F0895019110810EC0019104
:103230001191219130810BC00191108117FF05C0C0
:103240003FEF2FEF04C0008111272227332737FFDC
:1032500003C0E1DF8DE28D93CF93DF93CF92DF92B6
:10326000EF92AA24BB24CC24DD24EE2440E2CAE061
:10327000DD2755E093E38881890F87FD9F7083FDEB
:10328000907F891B89935A95A9F7C0DFAA1CBB1CA4
:10329000CC1CDD1CEE1C4A9551F7E894EFE0FF27AB
:1032A00082910ED0EB30E0F71EF068948A2D0CD09E
:1032B00088278D93EF90DF90CF90DF91CF91089585
:1032C000982F829501D0892F8F70805D26F08033F2
:1032D00009F4089568948D93089588278D9308952F
:1032E00081918D938823E1F7089594E081918D93E6
:1032F0009A95E1F7089509919191992351F08A9552
:10330000D9F7319781918D930A9519F08823D1F7D8
:103310000895E3CFFF935527F8E0469508F4500F42
:1033200057954795FA95D1F7FF910895FF93881B1C
:10333000F9E0001FFA9511F4FF910895881F841B8E
:1033400018F4840F8894F5CF0894F3CF8FEF83950A
:103350009D919923E1F708950DDD0F7708950ADD1A
:1033600013DD0395AAF087E1DD0CEE1CFF1C8A95A6
:1033700089F00A95CAF7FF205AF000240D280E287C
:103380000F28002039F00A95DD0CEE1CFF1CDAF73F
:103390000A950CCD98CDEEDC85E041D10F7723E87E
:1033A00039EF42E25EE3B1DDDBDF39DD139727D091
:1033B0008A3F40F000688D3F18F4E1DD80E803C0EB
:1033C00057D1E3DD882784832FDD9FDD28DD139728
:1033D00029EA3EE64CE952EC98DD22E332E541E889
:1033E00052E40AD122ED32EE4DE951EC05D120E94B
:1033F0003FEF4FE75FE3C9DD848108271DC1802FC0
:103400009F2D991F881F991F881F08955CCDB2DCDE
:103410000023E2F334DE19F44FDD0068089585E0FF
:10342000FED0FF0C001F04830FE70695F79420D110
:103430005068ABDDF4DC139721E438E743ED5BEB38
:1034400064DD27E831ED43E15DE3D6D02EE03CE3D7
:1034500043EC5DEBD1D022E83DEA4BE25EE3CCD019
:103460002CEE32E846E75EEBC7D020E931EE49EAC0
:103470005EE3C2D020E83FEE4FEF5EEBBDD024EC20
:103480003FEF4FE75FE3B8D0CADC139784818F57D3
:1034900099F02AF4D82E0FEFE02EF02E04C0D82E8B
:1034A000EE24FF2400278ADC28E132E741E35FE3D2
:1034B0002CDD65DC349769DDBFC05CDC80E003C0D7
:1034C00059DC802F8078882321F0DF92EF92FF92E1
:1034D0000F938F9359DC802F839512F4F4DC1BC07B
:1034E00080958A95885E0AF415C088501AF40CD02D
:1034F000D92210C0DD2488501AF406D0E9220AC06F
:10350000EE2402D0F92206C09FEF8770990F8A95AA
:10351000EAF708954BDC8F918823D9F35F914F919F
:103520003F912F910F9395DD0F9199F390F3A0D0D8
:1035300050682BCDC1DC80C01DDC86E070D00583D7
:103540000F772BE33AEA48EB5FE3DFDC68DC1397A5
:1035500041D028F4858188236AF7B5DC6DC08F7768
:10356000848308DC3497FCDE5ADC139723E632E4CC
:1035700046E357EBCADC29ED37EA4AE159E33CD090
:1035800026E538E14EEA5AEB37D026E53CE84DE136
:103590005CE332D02DEC37E543E65DEB2DD02DEE2C
:1035A0003DEF45E75EE328D028E132E741E35FEBFA
:1035B00023D05ED0EADC38DCDD24EE24FF24048155
:1035C0008FE7080F0695F7944ADC8581881F08F479
:1035D00038DC32C0D9DB8827039512F4889408952B
:1035E00007301AF0812F08940895FF1C881F0A9550
:1035F000E2F7812B88940895C8DCC1DB349785CC31
:10360000B9DB0F93AF93BF930F7702DFFF91EF9179
:10361000B6DB7BDC92DF8F918078082B08950FB6A4
:10362000F8944A925A92E42DF52DA42DB52D480E0A
:103630008827581E0FBE08950FB6F89459904990E8
:103640000FBE089597DB002331F02BED3FE049ECEE
:103650005FEB9BDCA1CE37CC8DDB802FFF0C001FF6
:10366000901728F4091B881F0795F79408952BCC11
:103670005FE340E83327222708957CDB0F930F7721
:103680007EDC1FDF8F918078082B08951CCC72DBC5
:103690000023E2F3D9F388E0C2DFC1DB1196FF0C0F
:1036A000001F8FE7080F0795F7940695F79483E0BE
:1036B0008F93BADBB4DB13975DDBD1DB60DB38972C
:1036C00064DC91E0CADF8F918A9511F08F93F1CF7E
:1036D000B3CF0000E4420AD71F4100000000000001
:1036E00020C100007A440000C842FB3A703D00004F
:1036F000F0415839343E0000A04100002041000054
:10370000803F1B2F654200000040000048423F2FD1
:103710005E76202E2D402526303132333435363733
:1037200038394142434445464748494A4B4C4D4E3F
:103730004F505152535455565758595A0000202053
:103740002020202020202020202020202020202079
:10375000000020484920000020002D2D2D2E2D0096
:103760002E2E2E2E2E00260025004000480033006D
:1037700032003100495733484556202F20504133FD
:10378000434B5200414E54454E4E4120414E414C18
:0C37900059534552000056302E323300D1
:00000001FF
